:0200000480007A
:100000006F004005732F2034930F8000630AFF03B5
:10001000930F90006306FF03930FB0006302FF038A
:10002000170F0000130F0F2463040F0067000F0069
:10003000732F203463540F006F00400093E19153FD
:10004000171F000023203FFC171F0000232E0FFA6C
:100050006FF01FFF930000001301000093010000E8
:10006000130200009302000013030000930300003A
:100070001304000093040000130500009305000022
:10008000130600009306000013070000930700000A
:1000900013080000930800001309000093090000F2
:1000A000130A0000930A0000130B0000930B0000DA
:1000B000130C0000930C0000130D0000930D0000C2
:1000C000130E0000930E0000130F0000930F0000AA
:1000D000732540F16310050097020000938202012E
:1000E000739052307350447497020000938202015F
:1000F00073905230735000189702000093820202EE
:1001000073905230B70200809382F2FF7390023BEB
:100110009302F0017390023A73504030970200004E
:1001200093824201739052307350203073503030BC
:100130009301000097020000938202ED7390523009
:10014000130510001315F501634C05000F00F00FA7
:10015000930110009308D005130500007300000000
:1001600093020000638A020073905210B7B200003D
:100170009382921073902230735000303725000024
:100180001305058073200530970200009382420119
:1001900073901234732540F17300203093012000D6
:1001A000B70703049387172097200000938080E50A
:1001B00003A70000B703030493831320631A770691
:1001C00093013000B707040593872730972000007C
:1001D000938040E303A71000B70304059383233003
:1001E0006318770493014000B707050693873740EB
:1001F00097200000938000E103A72000B7030506C5
:10020000938333406316770293015000B7070607C4
:1002100093874750972000009380C0DE03A73000EB
:10022000B7030607938343506314770063103002CB
:100230000F00F00F638001009391110093E1110012
:100240009308D00513850100730000000F00F00F24
:10025000930110009308D0051305000073000000FF
:100260009302400073232034E39462FC1387070059
:10027000F3221034938242007390123473002030C2
:10028000731000C00000000000000000000000002B
:10029000000000000000000000000000000000005E
:1002A000000000000000000000000000000000004E
:1002B000000000000000000000000000000000003E
:1010000000000000000000000000000000000000E0
:1010100000000000000000000000000000000000D0
:1010200000000000000000000000000000000000C0
:1010300000000000000000000000000000000000B0
:081040000000000000000000A8
:1020000001020304050607080000000000000000AC
:040000058000000077
:00000001FF
